:100000000C9434040C9451040C9451040C94510439
:100010000C9451040C9451040C9451040C9451040C
:100020000C9451040C9451040C9451040C945104FC
:100030000C9451040C9451040C9451040C945104EC
:100040000C9451040C9451040C9451040C945104DC
:100050000C945104167A0A0C20600001030705096C
:100060000701030305050103010305030505050554
:10007000050505050101050605050B070607070629
:10008000050707010507060707070607070607070D
:10009000070B07070702030205070205050405050C
:1000A000030505010205010905050505030503050D
:1000B000050905050503010306077F100700070072
:1000C000000024E43CE73C2724001000100000005E
:1000D000CE11FF11E200103010000E1111CE38E6E3
:1000E0001110E0000010000000101000E01E1129A7
:1000F000C6A000001010100000100700F806010054
:1001000030400106F8403000020A070A02000000F1
:10011000000010107C101000000000000070202073
:10012000200000000010807C03100000FE0101018F
:10013000FE00101010000402FF0000100281413187
:100140000E101010101082011111EE00101010008E
:10015000605846FF4000000010009C0B0909F100A8
:1001600010101000FE110909F2001010100001C15A
:100170003905030010000000EE111111EE001010FF
:1001800010009E212111FE001010100004100470B8
:1001900010282828440000000000484848484848E3
:1001A0000000000000004428282810000000000083
:1001B000060161110E0000100000F00CE2120909A6
:1001C000F119028678102040909090909050402035
:1001D00080702E212E708010000000000010FF1192
:1001E000111111EE1010101010007C82010101821B
:1001F0004400001010100000FF01010101827C107A
:10020000101010100000FF1111111111101010101A
:100210001010FF1111110110000000007C8201017B
:1002200011927400001010100000FF101010101038
:10023000FF10000000000010FF10C0000000FF00D1
:1002400010101000FF201028448201100000000050
:100250000010FF0000000000101010101010FF062A
:1002600078807806FF10000010000010FF020C10CC
:100270006080FF100000000000107C8201010182FC
:100280007C00001010100000FF111111110E100061
:10029000000000007C82014141827C0000101010AF
:1002A0000010FF11111131D10E10000000000010DC
:1002B000CE11111111E6001010101000010101FF04
:1002C000010101000000100000007F80000000809C
:1002D0007F00001010100000031C6080601C0300F1
:1002E000000010000000077880700E010E70807C06
:1002F00003000010000000000010000001C62810DC
:100300006C820110000000000010010608F00806D1
:100310000100000010000000008161110D030110B8
:10032000101010101010FF017040037C80000010AE
:1003300001FF4070100E010E1000000000000000D0
:1003400000000000004040404040404001020000EA
:10035000C82424A4F80010100010FF880404F8102A
:1003600000101000F804048800101000F80404883D
:10037000FF0010100010F8242424B8001010100002
:1003800004FE05001000F8040488FC405050403082
:10039000FF080404F81000000010FD1000FD4030BC
:1003A000FF2030C8041000000010FF10FC080404F7
:1003B000F8080404F8100000001000000010FC0809
:1003C0000404F81000000010F8040404F8001010F1
:1003D0001000FC880404F87000101000F804048871
:1003E000FC0010100070FC08041000009824242465
:1003F000C8001010100004FF04001010FC00008062
:10040000FC00101000100C7080700C000010000038
:100410000C7080700C7080700C00001000000010D8
:10042000000004D860980410000000100C70807068
:100430000C004030000004C4241C041010101010E4
:1004400020DE01003040FF7001DE2040300020102F
:1004500010202010000000000000FE020202020234
:10046000FE1010101010101000788078000008FEA8
:10047000000080007C82827C000000000000000000
:10048000000000000000000000000000000000006C
:10049000000000FC24241800E01010E000F000F040
:1004A00000F000E050506000F02010E0505060007C
:1004B000E010A0FC000000FC2424D80030C0300074
:1004C0000000000000000000000000003844BAAA4C
:1004D00044380000C4A2928C007C82827C00000818
:1004E000FE00007C82827C00000000000000000012
:1004F00000000000000000000000000000000000FC
:1005000000000000000000000000000000000000EB
:1005100000000001000000000001010000000100D7
:1005200001000000010101000100000001010100C3
:1005300000010001000000010101000004030000AF
:1005400000000000000000000000000000000000AB
:10055000000000000000000000000000000000009B
:10056000000000000000000000000000000000008B
:10057000000000000000000000000000000000007B
:1005800000000000000000027EFEFE0606068CFC55
:10059000F8F020E0E06060C0800000808080000013
:1005A00000000000000080F0FC7C1E0E0E1E0E06F7
:1005B0000002067EFEFE0E0E0E0E0E1E0E0C3EFEFF
:1005C000FEE0E0FEFE7E1C080000000000000000CF
:1005D000000000000000000000000000000000001B
:1005E000000000000000000000000000000000000B
:1005F00000000000000000000000000000000000FB
:10060000000000000000000000FFFF1C0E0E0703AA
:10061000010000FFFF187CC703FEFF030103FFFE7C
:100620000000000000007FFFFF80003C1C1CFCFC61
:1006300000000000FFFF06060E0E0602000000008C
:10064000F37F3FFB8000000000000000000000007E
:10065000000000000000000000000000000000009A
:10066000000000000000000000000000000000008A
:10067000000000000000000000000000000000007A
:100680000000000000000000001F1F00000000002C
:10069000000000070700000106000307060703002B
:1006A0000000000000000003070F1E1C1C0E7F004E
:1006B000000000001F1F00000000000000001807DD
:1006C000010000000718000000000000000000000A
:1006D000000000000000000000000000000000001A
:1006E000000000000000000000000000000000000A
:1006F00000000000000000000000000000000000FA
:100700000000F800F008F000F800F800F008F00031
:10071000F800F800F008F000F80000000000FF11F9
:1007200011110E00F81008F00808F000007C82019A
:100730001111F60000FF1111110101C62838C60180
:10074000000000F00808F000F81008F00890F80029
:100750000000000000000000000000000000000099
:100760000000000000000000000000000000000089
:100770000000000000000000000000000000000079
:100780000000000100000001000000C140404001E5
:10079000000000010000000100000001C000010095
:1007A000C0404040010000000101000000000001C5
:1007B00001010000C0010000C040414000000001F4
:1007C0000001000001010000010000040504030015
:1007D0000000000000000000000000000000000019
:1007E0000000000000000000000000000000000009
:1007F00000000000000000000000000000000000F9
:1008000000000000000000000000001F02020200C3
:100810000F10081F001F02011E0000007F000000D3
:100820001F020202001F02010E151516000E1515FB
:10083000160000007F0000001F121212001D151587
:100840001E0012150D00433C0300000000000000D4
:100850000000000000000000000000000000000098
:10086000000000000000000011241FBECFE5D8E00A
:10087000DEBFCDBF10E0A0E6B0E0EAE9F6E102C0DD
:1008800005900D92A037B107D9F714E0A0E7B0E0CA
:1008900001C01D92A237B107E1F70E9453040C94E6
:1008A0004B0B0C9400000E94FE0984E590E00E942E
:1008B0001F0B80E690E061E00E949D090E94C10943
:1008C0000895362F3770669566956695E62FFF2753
:1008D000F695FE2FEE27F795E795E80FF11DEE58F8
:1008E000FF4F2081413051F081E090E002C0880F3D
:1008F000991F3A95E2F78095822308C081E090E045
:1009000002C0880F991F3A95E2F7822B80830895E1
:10091000EF92FF920F931F93E22E480F87FD14C0B2
:10092000062F603408F00FE3413808F080E88417A0
:1009300068F4182FF42E4E2D602F812F0E94610431
:100940001F5FF116C1F702C08FE7EACF1F910F9129
:10095000FF90EF900895EF92FF920F931F93F82E60
:10096000E22E460F87FD14C0413470F060E4641736
:1009700090F4162F042F4E2D612F8F2D0E946104AD
:100980001F5F0117C1F707C0603488F36FE3EFCF33
:100990002FE7F22EE9CF1F910F91FF90EF9008956E
:1009A000BF92CF92DF92EF92FF920F931F93E82EA8
:1009B000D62EB42EC22E142F181B1F5FF22EF61A3D
:1009C000F394202F412F0E948804202F412F6C2D5B
:1009D0008E2D0E948804202F4F2D6D2D8E2D0E946C
:1009E000AB04202F4F2D6D2D8B2D0E94AB041F913A
:1009F0000F91FF90EF90DF90CF90BF900895CF922E
:100A0000DF92EF92FF920F931F93C62ED42EF22EF9
:100A1000E02E4817C0F02617B0F087FD14C047FD40
:100A200012C09FE3961778F0921768F0082F1C2DDC
:100A30004E2D612F802F0E9461041F5FF116C0F7B9
:100A40000F5FD016A0F71F910F91FF90EF90DF90EE
:100A5000CF9008950F9300E02FE34FE760E080E030
:100A60000E94FF040F9108954F925F926F927F92C0
:100A70009F92AF92BF92CF92DF92EF92FF920F932D
:100A80001F93CF93DF93CDB7DEB721970FB6F894BE
:100A9000DEBF0FBECDBFE42EF22EA02E481708F009
:100AA0004CC00FEF902EF61608F04CC0BFEFBB2ED7
:100AB0004E2D5527481B510957FD4CC02F2D33276C
:100AC000261B310937FD4FC0421753070CF452C0A3
:100AD0003901660C771C6901C41AD50ACC0CDD1CDF
:100AE0008E1509F48BC087FD92C0603408F08CC06D
:100AF0002301441A550A082F090DF82E162F0BC092
:100B00004C0C5D1C1B0DF90CE01689F007FD7FC035
:100B1000090D103470F44A2D612F8F2D0E9461044D
:100B200057FEEECF460C571CF90CE01679F7F7FC90
:100B30006EC0103408F06BC058C011E0912EF6164C
:100B400008F4B4CFA1E0BA2E4E2D5527481B510909
:100B500057FFB4CF509541955F4F2F2D3327261B5C
:100B6000310937FFB1CF309521953F4F42175307D9
:100B70000CF0AECF3A01660C771C6A01C21AD30A98
:100B8000CC0CDD1C6F15B9F187FD41C06034C8F590
:100B90002301421A530A162F1B0D082F962F0DC042
:100BA0004C0C5D1C090D9B0DF116A9F007FD2FC023
:100BB0001B0D812F8B19803480F44A2D692F802FD3
:100BC00099830E946104998157FEEACF460C571C15
:100BD0009B0DF11659F707FD1AC09034C0F44A2D49
:100BE000692F802F0E94610412C04A2D612F8F2D22
:100BF0000E9461040CC0082F962FEDCFF82E162FFF
:100C000096CF082F962FE9CFF82E162F92CF219648
:100C10000FB6F894DEBF0FBECDBFDF91CF911F910D
:100C20000F91FF90EF90DF90CF90BF90AF909F908B
:100C30007F906F905F904F9008958F929F92AF92A8
:100C4000BF92CF92DF92EF92FF920F931F93CF93B9
:100C5000DF93B82EA62EC22E282F3327642F772796
:100C6000C901860F971F803891050CF077C0261BAD
:100C7000370B37FD73C02A2D3327CB01820F931F0B
:100C8000803491050CF06AC0261B370B37FD66C017
:100C9000660F771FC3E0D0E0C61BD70BD42E882485
:100CA000992412C0882D99278D199109880F991FB1
:100CB000880F991F2A96C80FD91FDA940894811CAF
:100CC000911CED1408F04AC0E82CFD2CFA0C1B2DE9
:100CD000180D4C2D6F2D812F0E9461040A2D0D19C6
:100CE0004C2D602F812F0E9461041B2D18194C2D53
:100CF0006F2D812F0E9461044C2D602F812F0E9447
:100D00006104FA2CF80C1D2D1B0D4C2D6F2D812F1D
:100D10000E9461040A2D08194C2D602F812F0E941A
:100D200061041B2D1D194C2D6F2D812F0E94610414
:100D30004C2D602F812F0E946104D7FFB3CF882DE7
:100D40009927880F991F880F991F2696C80FD91FBA
:100D50000894811C911CED1408F4B6CFDF91CF915B
:100D60001F910F91FF90EF90DF90CF90BF90AF90C9
:100D70009F908F9008955F926F927F928F929F9233
:100D8000AF92BF92CF92DF92EF92FF920F931F9399
:100D9000CF93DF93582ED62EFA01C4903196A490AB
:100DA0003F010894611C711C8C2C9924C401850D91
:100DB000911D813891050CF047C0262F2A0D312D49
:100DC000311D213431050CF03FC0AA2009F43CC08C
:100DD000BB24CC20A9F18B2D8695869586959927E5
:100DE000889E7001899EF00C989EF00C1124E60CF0
:100DF000F71CCB2DDD27C770D070052D10E009C082
:100E000041E06D2D802F0E9461041F5F0F5FC116AE
:100E1000B9F0F701E10FF11DE4918E2F99270C2E07
:100E200002C0959587950A94E2F780FDE9CF40E0EE
:100E30006D2D802F0E9461041F5F0F5FC11649F75F
:100E4000B394D394AB1429F6DF91CF911F910F91F6
:100E5000FF90EF90DF90CF90BF90AF909F908F90DA
:100E60007F906F905F90089583E090E00E940C0B5C
:100E7000992787FD909508950F931F93082F84E07D
:100E800090E00E940C0B182F85E090E00E940C0B64
:100E9000011718F48FEF9FEF11C0202F3327810F18
:100EA000912D911D28173907ACF7011B802F992729
:100EB00006960E940C0B992787FD90951F910F9124
:100EC00008951F93CF93DF93EC0188818823A1F0CD
:100ED00010E006C0180F1F5F21968881882339F023
:100EE0000E943C078F3FB1F78FEF9FEF07C0812F24
:100EF000992787FD909502C080E090E0DF91CF9127
:100F00001F9108952F923F924F925F926F927F921E
:100F10008F929F92AF92BF92CF92DF92EF92FF9209
:100F20000F931F93CF93DF93CDB7DEB728970FB6FC
:100F3000F894DEBF0FBECDBF382EF62E042F222E22
:100F400083E090E00E940C0B8B8384E090E00E9491
:100F50000C0B182F85E090E00E940C0B011718F481
:100F60008FEF9FEF03C1202F3327A82EBB24C5018D
:100F7000810F911D281739079CF72B81822F992704
:100F80000796959587959595879595958795D82EEC
:100F9000011B09F4E4C08824992410E0812F9927CB
:100FA00006960E940C0B880E911C1F5F0117B1F76B
:100FB0002D2D33273D832C83289DC001299D900D25
:100FC000389D900D1124F5013696E80FF91FFA832C
:100FD000E983802F992706960E940C0BE82EF1E0FA
:100FE000DF1609F4B9C0AF2C442455243D2D3250EE
:100FF0003E83E49C4001112489819A81880E991EC8
:1010000061E0F62ECC24DD246A2C7724C601860DFF
:10101000971D8034910574F5EE2019F137FC21C03D
:10102000132D98868F8200E0BA2CBC0C0CC00F5F89
:10103000E016B9F01F5F17FD14C02F8138852F5FB0
:101040003F4F38872F838F8198850E940C0B8F210B
:1010500071F3422D6B2D812F0E9461040F5FE0160A
:1010600049F70894C11CD11C38E0C316D10411F013
:10107000FF0CCCCF88E0A80E0894411C511CEE81D7
:101080008E2F992701964816590609F0B2CF442DA4
:101090002C813D81220F331F220F331F220F331F5C
:1010A0003D832C838C813B81831B282F332778E061
:1010B000672E712C621A730A161417040CF049C0BB
:1010C0004A2C552480E4481651040CF042C081E0BB
:1010D00090E002C0880F991F2A95E2F7F82E4E9DE6
:1010E00040011124E981FA818E0E9F1ECC24EE204E
:1010F00019F137FC21C0132D98868F8200E0DA2C7D
:10110000DC0C0CC00F5FE016B9F01F5F17FD14C0B8
:101110002F8138852F5F3F4F38872F838F819885A8
:101120000E940C0B8F2171F3422D6D2D812F0E9497
:1011300061040F5FE01649F7C3948C2D992786153B
:1011400097053CF4840D951D8034910514F4FF0C33
:10115000CECF81E090E00AC0AF2C40E099CF80E094
:1011600090E0ED2DFF27FD83EC832DCF28960FB661
:10117000F894DEBF0FBECDBFDF91CF911F910F91CD
:10118000FF90EF90DF90CF90BF90AF909F908F90A7
:101190007F906F905F904F903F902F9008959F9217
:1011A000AF92BF92CF92DF92EF92FF920F931F9375
:1011B000CF93DF93CDB7DEB727970FB6F894DEBF96
:1011C0000FBECDBF982EA62EFA01422FB02E6E0173
:1011D0000894C11CD11C87E0D6011D928A95E9F7BD
:1011E000F7FD59C080E28F833097A1F096012B5F05
:1011F0003F4FCF016AE070E00E94240BD9018C932D
:1012000021503040CF016AE070E00E94240BFB01C6
:10121000672B79F74F3F99F1842F992787FD909598
:10122000A6E0EA2EF12CE81AF90A1F812B2D412F96
:101230006A2D892D0E948207812F0E943C07B6E00B
:10124000EB16F104F4F5082F0F5F090DCE0CDF1C2F
:10125000F60111916F01105D2B2D412F6A2D802F0A
:101260000E948207812F0E943C078F5F080F08941D
:10127000E11CF11CF6E0EF16F10454F322C0898161
:10128000882379F4F601818131968823E1F37F0187
:10129000EC18FD08CACF8DE28F83F095E195FF4FE2
:1012A000A3CF1F812B2D412F6A2D892D0E948207EC
:1012B000812F0E943C07082F0F5F090DEE24FF24A9
:1012C000C5CF27960FB6F894DEBF0FBECDBFDF9116
:1012D000CF911F910F91FF90EF90DF90CF90BF9033
:1012E000AF909F900895FF920F931F93CF93DF933A
:1012F000182FF62EEA01022F4881442361F415C00D
:1013000088810E943C078F3F69F0219648814423E1
:1013100061F08F5F180F202F6F2D812F0E948207A1
:101320008F3F71F78FEF9FEF02C081E090E0DF9178
:10133000CF911F910F91FF9008950F931F93CF931B
:10134000DF93EC01062F0E946107869510E4181BBD
:1013500017FF03C08FEF9FEF0FC00E9434078695E1
:1013600060E2681B6034B0F7202FAE01812F0E942D
:101370007309992787FD9095DF91CF911F910F9168
:101380000895CF92DF92EF92FF920F931F93CF9326
:10139000DF93B2E7EB2EB0E0FB2ECC24DD240C2D46
:1013A0000E94530A8C2D0E944D0AE70110E089919A
:1013B0000E942C0A1F5F1034D1F780E490E0E80E01
:1013C000F91E0E94560A802F0E944D0AF701819152
:1013D0007F010E942C0A1F5F1038C1F70894C11CBE
:1013E000D11CF8E0CF16D104D1F6DF91CF911F9137
:1013F0000F91FF90EF90DF90CF9008950E94D40A54
:101400000895C4989698939895E0292F2A95F1F716
:10141000C49A85BB9A95F1F7C498089514BA81E0EF
:101420008A95F1F725E031E0C498969A9398822F37
:101430008A95F1F7C49A822F8A95F1F783B3C498FD
:10144000932F9A95F1F787FDEFCF96988AE08A95CA
:10145000F1F78FEF84BB0895C4989698939A95E01E
:10146000292F2A95F1F7C49A85BB9A95F1F7C4986C
:101470000E940E0A08958FE30E94010A0E940E0A3C
:1014800008958EE30E94010A0E940E0A0895806466
:101490000E94010A0E940E0A0895886B0E94010AA8
:1014A0000E940E0A0895C198C09A0895C098C19AE2
:1014B0000895CF92DF92EF92FF920F931F93CF93F5
:1014C000DF937C01CC24DD240C2D0E94530A8C2D4B
:1014D0000E944D0AE70110E0FE012196E4918E2F53
:1014E0000E942C0A1F5F1034B9F780E490E0E80EE8
:1014F000F91E0E94560A802F0E944D0AF701089497
:10150000E11CF11CE4918E2F0E942C0A1F5F103801
:10151000A9F70894C11CD11C98E0C916D104A1F602
:10152000DF91CF911F910F91FF90EF90DF90CF90BF
:10153000089540E050E020E030E0FC010196E491A5
:101540004E0F511D2F5F3F4F64E020303607A9F743
:101550004E5C524709F0FFCF08950F931F93CF932E
:10156000DF93C0E0D0E00C2F0E94530A8C2F0E9422
:101570004D0A10E080E00E942C0A1F5F1034D1F762
:101580000E94560A802F0E944D0A80E00E942C0A79
:101590001F5F1038D1F72196C830D10521F7DF91B0
:1015A000CF911F910F9108958FEF84BBBC9A8E9AB3
:1015B0008B9AB89AB99A0E94530A0E940E0A0E9406
:1015C0003B0A80E00E94470A80E00E944D0A0E9488
:1015D000560A0E940E0A0E943B0A80E00E94470AB7
:1015E00080E00E944D0A88E694E00E94590A88E64D
:1015F00094E00E94990A20E0E0E0F0E0CF0101973A
:10160000F1F72F5F283CD1F70E94AD0A08950895A5
:10161000FC01849199270895209170003091710008
:10162000820F931F0E94080B9927089580917000E4
:101630009091710003960E94080B9927089590934A
:10164000710080937000089597FB092E07260AD039
:1016500077FD04D00CD006D000201AF47095619567
:101660007F4F0895F6F7909581959F4F0895AA1B97
:10167000BB1B51E107C0AA1FBB1FA617B70710F07D
:10168000A61BB70B881F991F5A95A9F780959095AF
:0A169000BC01CD010895F894FFCFCE
:10169A0048656C6C6F204772617068695821000058
:00000001FF
